:100000000C941E060C9450280C947D280C944606E3
:100010000C9446060C9446060C9446060C94460630
:100020000C9446060C9446060C942C130C9446062D
:100030000C9446060C9446060C9446060C94460610
:100040000C94AA280C9446060C94982C0C94DB2C47
:100050000C9446060C9446060C9446060C944606F0
:100060000C9446060C944606DB183D191C191F1902
:100070002219251928192B192E193D1937196F1A0C
:10008000711A711A6F1A711A711A711A711A711A1A
:10009000711A711A711A711A711A711A711A711A08
:1000A000F519711A711A711A711A711A6619711A81
:1000B000711A711A711A711A711A711A711A711AE8
:1000C000711A711A711A711A711A711A011A011AB8
:1000D000011A011A011A011A011A011A011A711AD8
:1000E000711A711A711A711A711A6619001A001AA6
:1000F000001A001A711A0E1A141A1A1A201A261A3D
:100100002C1A321A381A421A4C1A561A601AA7199F
:100110006919711A711A711A711AF519711A711A0D
:10012000711A711A711A711A711A711AFF19FF195D
:10013000FF19FF19711A0E1A141A1A1A201A261A00
:100140002C1A321A381A421A4C1A561A601AA7195F
:100150006919711A711A711A711AF519A41AA41A67
:10016000A41AA41AA41AA41AA41AA41AA41AA41A9F
:10017000A41AA41AA41ABA1BBA1BBA1BBA1BBA1B1C
:10018000BA1BE91AF31AFD1A071B641B6E1B7D1BB1
:100190008E1B161D2B1D371D401D4F1D741D7D1DF3
:1001A000C61D8F1DDB20E120E720EE20FC201E2154
:1001B0003C21456E746572206D656E752E2E2E0085
:1001C000546F67676C6564206D6963726F50504D42
:1001D00000546F67676C656420696E76657274653C
:1001E000642050504D2100546F67676C6564205443
:1001F00058206D7574696E672100546F67676C6570
:10020000642074656C656D65747279210050726F3D
:10021000746F636F6C206572726F72207769746897
:100220002052580054696D656F7574207768656E4B
:1002300020636F6E6E656374696E6720746F205201
:100240005800507265737320616E79206B65792058
:10025000746F2063616E63656C00436F6E6E6563DF
:1002600074696E6720746F2052582C20706F776508
:100270007220757020746865205258202877697440
:10028000682062696E6420706C7567206966206EF4
:100290006F74207573696E6720616C776179732064
:1002A00062696E642900546F67676C656420276912
:1002B0006D6D656469617465206F75747075742700
:1002C00000546F67676C65642027736C61766520E6
:1002D0006D6F64652700546F67676C6564202761E4
:1002E0006C776179732062696E642700546F676769
:1002F0006C65642050504D206368616E6E656C20A3
:100300006C696D69740053657420525353492069B8
:100310006E6A656374696F6E206368616E6E656C8A
:100320002028303D3D64697361626C652900536526
:10033000742050504D206D696E696D756D20737914
:100340006E630053657420626561636F6E20696E31
:1003500074657276616C0053657420626561636FC9
:100360006E2064656C617900536574206265616319
:100370006F6E206672657175656E637920696E2097
:10038000487A3A20303D64697361626C652C205074
:10039000783D504D52206368616E6E656C20782CFC
:1003A0002046783D465253206368616E6E656C202E
:1003B00078005365742050574D2073746F7020641B
:1003C000656C61792028302064697361626C6564B2
:1003D0002C20312D323535203D3D20302E317320FB
:1003E0002D2035306D696E29005365742050504DB5
:1003F0002073746F702064656C61792028302064EC
:10040000697361626C65642C20312D323535203D75
:100410003D20302E3173202D2035306D696E29003E
:10042000536574206661696C736166652064656CF0
:1004300061792028302064697361626C65642C20C6
:10044000312D323535203D3D20302E3173202D2089
:1004500035306D696E29002A2A2A2A2A2A2A2A2A50
:100460002A2A2A2A2A2A2A2A2A2A2A2A2A2A2A2AEC
:100470002A2A2A2A0052582041636B6564202D20C5
:1004800072657665727420737563636573736675E0
:100490006C21002A2A2A2A2A2A2A2A2A2A2A2A2AAD
:1004A0002A2A2A2A2A2A2A2A2A2A2A2A2A2A2A2AAC
:1004B000002A2A2A2A2A2A2A2A2A2A2A2A2A2A2AC6
:1004C0002A2A2A2A2A2A2A2A2A2A2A2A2A2A00528E
:1004D000582041636B6564202D20757064617465DC
:1004E000207375636365737366756C21002A2A2A0D
:1004F0002A2A2A2A2A2A2A2A2A2A2A2A2A2A2A2A5C
:100500002A2A2A2A2A2A2A2A2A2A0056616C696457
:100510002063686F69636573206172653A205B319F
:100520005D2D5B31365D20286368616E6E656C20E1
:10053000312D31362900536574206F7574707574D0
:1005400020666F7220706F727420005B585D2061AE
:10055000626F7274206368616E67657320616E6498
:10056000206578697420525820636F6E6669670051
:100570005B535D20736176652073657474696E6783
:100580007320746F205258005B525D20726576654F
:1005900072742052582073657474696E6773207486
:1005A0006F2064656661756C747300557365206EA9
:1005B000756D62657273205B312D445D20746F2010
:1005C0006564697420706F727473205B452D515D92
:1005D00020666F722073657474696E677300202DD6
:1005E00020726563656976657220636F6E66696700
:1005F000757261746F722C20727820737720000AF4
:100600000A6F70656E4C52536E67200053657420FC
:1006100073657269616C2062617564726174653AB8
:10062000200056616C69642063686F696365733A82
:100630002031202D20342B34202F2032202D203823
:10064000202F2033202D20382B34202F2034202D14
:10065000203132202F2035202D2031322B34202FF5
:100660002036202D20313600536574204368616E9A
:100670006E656C20636F6E6669673A20005365741F
:100680002044617461726174652028302D32293AEA
:10069000200053657420486F70206368616E6E653A
:1006A0006C7320286D61782032342C207365706162
:1006B000726174656420627920636F6D6D61732966
:1006C0002076616C69642076616C75657320312DCC
:1006D0003235353A2000536574206368616E6E656B
:1006E0006C2073706163696E6720287831306B48C5
:1006F0007A293A200053657420524620706F77653E
:10070000722028302D37293A200053657420524634
:10071000206D6167696320286865782920652E67E8
:100720002E20307844454144463030443A2000532E
:1007300065742062617365206672657175656E63AC
:10074000792028696E20487A293A20005B5A5D207A
:10075000656E746572207265636569766572206383
:100760006F6E66696775726174696F6E2075746902
:100770006C79005B465D20646973706C61792061FF
:10078000637475616C206672657175656E63696509
:10079000732075736564005B525D2063616C6375E3
:1007A0006C6174652072616E646F6D206B65792079
:1007B000616E6420686F70206C697374005B495DC2
:1007C000207265696E697469616C697A6520736508
:1007D0007474696E677320746F20736B65746368DB
:1007E0002064656661756C7473005B585D2072658A
:1007F00076657274206368616E67657320616E64EC
:100800002065786974206D656E75005B535D20739B
:100810006176652073657474696E677320746F20E8
:10082000454550524F4D20616E64206578697420B3
:100830006D656E7500557365206E756D62657273BA
:10084000205B302D395D20746F20656469742070E1
:100850006172616D657465727300202D2053797328
:1008600074656D20636F6E66696775726174696F18
:100870006E000A0A6F70656E4C52536E672000510D
:1008800029204F7574707574206265666F726520DB
:100890006C696E6B20283D465329203A2000502970
:1008A00020536C617665206D6F64652028657870D3
:1008B0006572696D656E74616C293A20004F29205C
:1008C00054696D65642042494E44206174207374FC
:1008D000617274757020203A20004E292050504DCE
:1008E000206F7574707574206C696D69746564200F
:1008F000202020203A200044495341424C454400E6
:100900004D292050504D205253534920746F20637D
:1009100068616E6E656C202020203A20004C2920F2
:1009200050504D206D696E696D756D2073796E63E1
:10093000202875732920203A200044495341424C15
:100940004544004B29204661696C736166652062ED
:100950006561636F6E20696E74762E2028312D32AA
:10096000353573293A20004A29204661696C736144
:10097000666520626561636F6E2064656C617920D5
:1009800028302D323535203D3E20313073202D204A
:100990003135306D696E293A200049292046616958
:1009A0006C7361666520626561636F6E206672714B
:1009B0002E203A200048292050574D2073746F7024
:1009C0002064656C6179202020202020203A2000BE
:1009D00047292050504D2073746F702064656C61FE
:1009E00079202020202020203A200046292046611E
:1009F000696C736166652064656C617920202020D4
:100A00002020203A200050574D206368616E6E65AB
:100A10006C200066756E6374696F6E3A2000292041
:100A2000706F72742000506F776572546F776572C3
:100A300000445446205548462033322D62697420C4
:100A400031306368004F70656E4C52536E67525878
:100A5000206D696E6920342F36636800466C7974A6
:100A6000726F6E2F4F72616E6765525820554846FF
:100A70002038636800525820747970653A20004429
:100A8000697361626C656400487A00203D3D200016
:100A900043616C63756C61746564207061636B6540
:100AA0007420696E74657276616C3A200042292068
:100AB0004D6963726F202868616C66292050504D23
:100AC000202020203A00412920496E766572746505
:100AD000642050504D20696E20202020203A0030A4
:100AE00029204D7574652062757A7A657220286DAB
:100AF0006F73746C79293A003929205365726961E2
:100B00006C2062617564726174653A00736D617224
:100B100074506F7274004672536B79005472616E38
:100B200073706172656E740044697361626C6564B0
:100B30000038292054656C656D657472793A2020FF
:100B40002020202020003729204368616E6E656CCC
:100B500020636F6E6669673A202000362920446161
:100B60007461726174652028302D32293A2020206A
:100B700000352920486F70206368616E6E656C7364
:100B80003A2020202020003429204368616E6E65C1
:100B90006C2073706163696E673A202000332920EE
:100BA000524620706F7765722028302D37293A2001
:100BB0002020003229205246206D616769633A2067
:100BC0002020202020202020003129204261736530
:100BD000206672657175656E63793A202020000089
:100BE00000000700020100000304060000000000EE
:100BF00000000001020408102040800102040810D7
:100C00002001020408102004040404040404040263
:100C10000202020202030303030303000000002395
:100C2000002600290000000000250028002B0000FD
:100C3000000000240027002A0000C92D11241FBE37
:100C4000CFEFD8E0DEBFCDBF13E0A0E0B1E0E0EA37
:100C5000F1E602C005900D92A83CB107D9F716E065
:100C6000A8ECB3E001C01D92A239B107E1F71CE086
:100C7000CCE3DCE004C02297FE010E94D22ECA33EE
:100C8000D107C9F70E94052E0C94CE300C940000B9
:100C900080917705813019F482E080937705809107
:100CA0007705833019F484E0809377050895A8953B
:100CB0000895DC01ED91FC910190F081E02D099502
:100CC00008952091780530917905382748E0C901C9
:100CD000880F991F37FF06C09C0151E2252750E17C
:100CE000352701C09C01415091F73093790520933D
:100CF0007805089588E380937A0580E092ECA1E07E
:100D0000B0E080937B0590937C05A0937D05B09324
:100D10007E0587E08093870580E091EAACEBB3E342
:100D200080937F0590938005A0938105B093820501
:100D300085E0809388058DEE9EEFADEABEED809351
:100D4000830590938405A0938505B0938605E9E813
:100D5000F5E080E090E0863028F4DC01AE54BC4F32
:100D60002C9101C020E0219301968831910599F7DB
:100D700082E08093A1058AE08093A205089580E037
:100D80009EECADEEB4E38093BF059093C005A093B5
:100D9000C105B093C20580E090E0A0E0B0E580938B
:100DA000C3059093C405A093C505B093C605E7ECB1
:100DB000F5E080E081938F5F8031E1F70895A0E056
:100DC000B0E0E5EEF6E00C949B2ED82F0E940029AF
:100DD0006115710581059105C9F30E943E2F10929E
:100DE0008305109284051092850510928605C4E053
:100DF000812C912C54018A94C0908305D090840555
:100E0000E0908505F0908605FE2CED2CDC2CCC24A2
:100E10000E94392FA50194010E947A2E6C0D7D1D30
:100E20008E1D9F1D609383057093840580938505B7
:100E300090938605C15001F7DD2309F450C009E8FD
:100E400015E0E801A12CB12C62E3C62ED12CE12CD7
:100E5000F12C8881882309F442C0B39419F40E94CC
:100E60007A063DC00E94392FA70196010E947A2E72
:100E7000E1E0E60FA9E8B5E08A2F801B8A1520F48F
:100E80008D918E13F9CFE9CF2091880530E0A0E154
:100E9000B7E20E94122E9B01AC01AE2FB0E00E947F
:100EA000212E40907F0550908005609081057090C4
:100EB0008205640D751D861D971D4090BF055090DD
:100EC000C0056090C1057090C205461657066806B9
:100ED000790618F2E993A39488E1A812BACFCDB7A6
:100EE000DEB7E0E10C94B72E8436910520F4BC0106
:100EF00080E090E017C09C018E3B910528F42A55B4
:100F00003109AAE0B0E00CC0823D910528F4245BD1
:100F10003109A4E6B0E004C02D5C3109A8E5B2E0D7
:100F20000E94122EA4E6B0E09B01AC010E94212E8B
:100F3000089590E08C599F4F0E947407089561E0D6
:100F400083E10E94AD2960E083E10E94E62982E00E
:100F50008093B00085E08093B10061E083E00E945F
:100F6000AD2960E083E00E94E6290895A4E0B0E0A6
:100F7000ECEBF7E00C94A92E009749F19C0140E0BE
:100F800050E068E478EE81E090E00E947A2E61E023
:100F900083E129833A834B835C830E94E62929817C
:100FA000822F3A81932F4B81A42F5C81B52F8F3FE5
:100FB0009105A105B10529F020F08FEF90E0A0E0A8
:100FC000B0E08093B3008091B000806107C060E022
:100FD00083E10E94E6298091B0008F7E8093B0006B
:100FE0002496E2E00C94C52E60E08CE00E94AD29CE
:100FF00061E08BE00E94AD2961E08DE00E94AD29A7
:1010000060E082E00E94AD2961E084E00E94AD29A9
:10101000089542E050E068E476E080E00E943028E5
:101020000895E3E0F0E089E080935700E491E670F2
:1010300081E0E63009F080E00895CF93DF93C82F78
:101040000E941108882381F0DFB781E08093760544
:10105000F8940E94570688E180936000C093600076
:10106000C1110E945706DFBFDF91CF9108958F9283
:101070009F92AF92BF92CF92DF92EF92FF92CF9367
:10108000FC01C0A5EC2FE770F0E0E658FC4FA08112
:10109000B0E0C7FF03C024E130E002C02FE030E041
:1010A000FC0197A183E1989FF0011124E25CFE4FBF
:1010B00080809180A280B380A20FB31F20E43FE123
:1010C0004DE750E00E942C2EA50194010E94582E5D
:1010D0008C2F887149F469017A01E0EDCE0EE7E0CA
:1010E000DE1EE11CF11C1BC0C7FF05C060E47AE8EE
:1010F0008CE29EE004C060E07EEE8AEB9BE069013A
:101100007A01F8EBCF0EFBE0DF1EE11CF11CA5011C
:1011100094010E94582EC20ED31EE41EF51EC70174
:10112000B60169517C4F8F4F9F4F28EE33E040E06E
:1011300050E00E94582EA8EEB3E00E94212ECF91DD
:10114000FF90EF90DF90CF90BF90AF909F908F90E7
:1011500008958F3F910551F048F0811522E09207E4
:1011600038F08115934030F482E0089580E00895CE
:1011700081E0089583E00895A0E0B0E0E2ECF8E0BB
:101180000C94A42EEB018A01B82FB695A0E028811B
:101190003981F80120832A813B8121832C813D8183
:1011A00022832E813F812383688179814A815B81FB
:1011B0002C813D81EE81FF819F2F9295990F990F90
:1011C000907C272F2370922B252F2370220F220F24
:1011D000922B232F23702295207F922BF80194834A
:1011E0000B5F1F4F2896AF5FBA1788F680FF24C0A9
:1011F000888199810E94A908D82E8A819B810E94AA
:10120000A908E82E8C819D810E94A908F82E8E8164
:101210009F810E94A908F0E4DF9EA001112490E1C3
:10122000E99E90011124242B282BE4E0FE9EB001BE
:101230001124262BF8012083CDB7DEB7E7E00C940C
:10124000C02E803223E0920708F1883E23E0920707
:1012500040F48F519340E4E096958795EA95E1F745
:101260000895803D27E0920718F48C5D934008951F
:10127000883928E0920768F4885C974074E0969576
:1012800087957A95E1F78D509C4F089580E090E026
:1012900008958FEF93E008958C30910540F4A4E019
:1012A000880F991FAA95E1F7885D9C4F0895843FA8
:1012B00023E0920718F484529C4F0895811524E08E
:1012C000920740F48657934FF4E0880F991FFA95E0
:1012D000E1F7089580E998E008959C0136952795F7
:1012E00025753575821B930B9C012373337396957B
:1012F00087959695879583739373820F931F9C01AF
:1013000054E0369527955A95E1F7280F391F2F702D
:101310003F7041E051E0249FC001259F900D349F14
:10132000900D1124892F08952D98882319F000001D
:101330002B9A02C000002B9800002D9A00000895FF
:101340002D9A000083B12D98000082958170089538
:10135000CF93DF93D82F5C9A2D985C98C8E08D2F9F
:1013600080780E949409DD0FC150C9F72D98DF9154
:10137000CF9108958F770E94A8090895CF93DF93A6
:10138000D82FC8E08D2F80780E949409DD0FC150BE
:10139000C9F72D98DF91CF910895CF93DF932D98C2
:1013A000C8E080E0D82FDD0F0E94A0098D0FC1504A
:1013B000C9F7DF91CF9108950E94BA090E94CD0923
:1013C0005C9A0895A1E0B0E0E8EEF9E00C94A92E53
:1013D000806869830E94A8096981862F0E94BE09DE
:1013E0005C9A2196E2E00C94C52ECF93C0918305C0
:1013F000C827E82FF0E0E658FA4F678589E70E9492
:10140000E2096C2F8DE30E94E2096C2F82E40E94B6
:10141000E209CF91089586E20E94DC090895CF93F6
:10142000DF93EC016C818CE10E94E2096D818DE11A
:101430000E94E2096E818EE10E94E2096F8180E2E2
:101440000E94E209688581E20E94E209698582E2E0
:101450000E94E2096A8583E20E94E2096B8584E2C8
:101460000E94E2096C8585E20E94E2096D858AE2AC
:101470000E94E2096E858EE60E94E2096F858FE682
:101480000E94E209688980E70E94E209698981E790
:101490000E94E2096A8982E70E94E209DF91CF9106
:1014A0000895CF92DF92EF92FF92CF93DF936B017B
:1014B0007C01C11488E3D8068CE9E8068CE1F806C3
:1014C00028F5C701B60120E836E948E950E00E9456
:1014D000582EE901689760E879E687E69FEF0E9459
:1014E000342E6C0D7D1D8E1D9F1DF2E0660F771F43
:1014F000881F991FFA95D1F721E732E040E050E0CC
:101500000E94582EF22EE32E80E421C0C701B601BE
:1015100020E03DE241E351E00E94582EE901689746
:1015200060E073ED8EEC9EEF0E94342E6C0D7D1DFD
:101530008E1D9F1D660F771F881F991F21E732E0C0
:1015400040E050E00E94582EF22EE32E80E66C2FF1
:101550006F71680F85E70E94E2096E2D86E70E9491
:10156000E2096F2D87E70E94E209DF91CF91FF909A
:10157000EF90DF90CF900895682F8DE60E94E209EA
:1015800008958F929F92AF92BF92CF92DF92EF9287
:10159000FF92CF93DF93D82F83E00E94DC098093E2
:1015A000750584E00E94DC098093740560E086E0A4
:1015B0000E94E20961E087E00E94E2096FE789E0AA
:1015C0000E94E20965E08AE00E94E20962E18BE0A4
:1015D0000E94E20965E18CE00E94E2096DEF8DE076
:1015E0000E94E20960E08EE00E94E209DD2319F02A
:1015F0008BE291E008C02091A10533E1239FC00157
:101600001124825C9E4F0E940F0A6CE880E30E94C6
:10161000E2096FE082E30E94E20962E483E30E9450
:10162000E2098091A20587FF02C064E101C06AE07F
:1016300084E30E94E2096AE285E30E94E2096DE226
:1016400086E30E94E20964ED87E30E94E20960E01C
:1016500088E30E94E20960E089E30E94E209D11177
:1016600009C0C0908305D0908405E0908505F09076
:10167000860507C0C5E9CC2EC1ECDC2EED2CCEEDE5
:10168000FC2ECAE38F2C9924AA24BB24682D8C2F0E
:101690000E94E209682D85E08C0F0E94E209FE2C71
:1016A000ED2CDC2CCC24CF5FCE3361F76FEF83E4DD
:1016B0000E94E2096FEF84E40E94E2096FEF85E483
:1016C0000E94E2096FEF86E40E94E209DD2311F037
:1016D00066E002C0609187058DE60E94E20960E045
:1016E00089E70E94E209609188058AE70E94E20981
:1016F00060E083E70E94E20960E084E70E94E2097B
:10170000D11109C060917F0570918005809181059C
:101710009091820504C060E071EA8CEB93E30E9433
:10172000510ADF91CF91FF90EF90DF90CF90BF9063
:10173000AF909F908F90089561E087E00E94E2094A
:1017400064E28EE70E94E20963E088E00E94E20919
:1017500060E088E00E94E20965E087E00E94E2091B
:1017600062E085E00E94E20983E00E94DC09809348
:10177000750584E00E94DC0980937405089583E078
:101780000E94DC098093750584E00E94DC09809347
:10179000740561E087E00E94E2096AE070E080E0A1
:1017A00090E00E9423290E949C0B00000895CF9294
:1017B000DF92FF920F931F93CF93DF931F92CDB7CA
:1017C000DEB7082F162F8EE399830E94E209F02ED0
:1017D000C02E9981D92E8C2D8F19811738F4F601DE
:1017E00061916F018FE70E94E209F5CF64E085E027
:1017F0000E94E20983E00E94DC098093750584E081
:101800000E94DC09809374050E9400296093700592
:1018100070937105809372059093730569E087E07A
:101820000E94E20981E0809377050F90DF91CF91CC
:101830001F910F91FF90DF90CF9008950F931F930A
:101840000E94D70B80917705813099F40E9400297E
:10185000009170051091710520917205309173050A
:10186000601B710B820B930B603A764881409105A7
:1018700048F380917705813031F46EE971E086EEAE
:1018800095E00E94EC2A1F910F9108950F931F93EA
:1018900080917705823021F41092770581E020C095
:1018A000809177058130D9F40E940029009170055C
:1018B000109171052091720530917305601B710BB9
:1018C000820B930B613A76488140910540F061E0CC
:1018D00087E00E94E2091092770582E001C080E073
:1018E0001F910F910895CF93DF93EC014AE050E0F0
:1018F0006D2F70E086EE95E00E94BA2B6EE286EEC8
:1019000095E00E94BE2ABE0184E0769567958A958F
:10191000E1F76F7077274AE050E086EE95E00E948D
:10192000BA2B6EE286EE95E00E94BE2ABE016F7071
:1019300077274AE050E086EE95E00E94BA2BDF91CF
:10194000CF910895D82FC0E0CD1780F4439A64E674
:1019500070E080E090E00E942329439864E670E004
:1019600080E090E00E942329CF5FEECF6CE271E02F
:1019700080E090E00E942329E6CF0F931F93CF933E
:10198000DF93EC01062F15E0115051F0CE010E94BB
:10199000B530081741F0602FCE010E94BD30F4CF62
:1019A00082E00E94A20CDF91CF911F910F910895C8
:1019B000A0E0B0E0EEEDFCE00C949B2E482E562EFD
:1019C000C0E0D0E0612C712CE12CF12C00E010E0A3
:1019D00041100CC06090D80586E4689E3001112447
:1019E00059E1E52EF12C0EEB15E01EC091E04912F5
:1019F0000FC06090D805E6E46E9E30011124FBE133
:101A00006F0E711C49E2E42EF12C0AE715E00CC0C0
:101A100082E0481209C028E1622E77247394EE24F4
:101A2000E394F12C07ED15E043018C0E9D1E1092FE
:101A30007905109278053401A62CA818B12CC301A1
:101A400001966C01AE14BF04A8F4A00EB11E511093
:101A500006C0C3010E94B530F501808305C0F501C1
:101A60006081C3010E94BD0CF50180810E94610666
:101A70003601E2CFC301511018C0C3010E94B53036
:101A8000B82EC6010E94B5302B2D30E0322F222710
:101A9000282B80917805909179058217930779F426
:101AA000C0E0D0E05524539493CF3601609179057E
:101AB0000E94BD0C60917805C6010E94BD0CC05EFD
:101AC000DE4FC13E92E0D90708F482CF852DCDB715
:101AD000DEB7E0E10C94B72E61E082E00E94D80C02
:101AE000089560E082E00E94D80C8091D70585308F
:101AF00020F01092D7050E946C0D8091D70580933D
:101B0000D805089561E080E00E94D80C61E081E092
:101B10000E94D80C089560E080E00E94D80C8823D1
:101B200051F060E081E00E94D80C882321F0809180
:101B30007A05883349F00E94BF060E947A0681E048
:101B40000E94DF060E94820D0895882319F06AEA38
:101B500071E002C06EEA71E086EE95E00E94EC2A28
:101B60000895FF920F931F93CF93DF9369EC7BE06F
:101B700086EE95E00E94982A40917F05509180055D
:101B800060918105709182052AE030E086EE95E053
:101B90000E94C12B63EB7BE086EE95E00E94982AC1
:101BA000409183055091840560918505709186056B
:101BB00020E130E086EE95E00E94C12B6DE97BE0EC
:101BC00086EE95E00E94982A4AE050E060918705F1
:101BD00086EE95E00E94E92B67E87BE086EE95E0D3
:101BE0000E94982A4AE050E06091880586EE95E0D0
:101BF0000E94E92B61E77BE086EE95E00E94982A3F
:101C0000C9E8D5E0F12C8E0188818823A9F0FF2056
:101C100031F061EB71E086EE95E00E94BB2A2196DF
:101C20004AE050E0F801608186EE95E00E94B22B18
:101C3000F394F8E1FF12E7CF86EE95E00E94C62A02
:101C40006BE57BE086EE95E00E94982A4AE050E042
:101C50006091A10586EE95E00E94E92B66E47BE0A9
:101C600086EE95E00E94982AE091A205E770F0E0E8
:101C7000EE0FFF1FEE57FC4F6081718186EE95E0FD
:101C80000E94EC2A61E37BE086EE95E00E94982AB0
:101C90008091A2058871883069F028F4811113C001
:101CA00068E27BE00CC0803141F0883161F46CE087
:101CB0007BE005C06CE17BE002C066E17BE086EE84
:101CC00095E00E94DA2A68EF7AE086EE95E00E94BD
:101CD000982A40917B0550917C0560917D0570911B
:101CE0007E052AE030E086EE95E00E94C12B6FED84
:101CF0007AE086EE95E00E94982A8091C305807173
:101D00000E94A50D66EC7AE086EE95E00E94982A86
:101D10008091C30580740E94A50D6DEA7AE086EE7D
:101D200095E00E94982A8091C30580720E94A50DBB
:101D300060E97AE086EE95E00E94982A8AE795E0CD
:101D40000E943708AB01BC012AE030E086EE95E046
:101D50000E94A32B6BE87AE086EE95E00E94982A19
:101D60008AE795E00E9437089B01AC0160E472E4C9
:101D70008FE090E00E94582EBA01A9012AE030E0DD
:101D800086EE95E00E94A32B68E87AE086EE95E067
:101D90000E94DA2ACDB7DEB7E5E00C94C22E8F920E
:101DA0009F92AF92BF92CF92DF92EF92FF928111FA
:101DB00007C06FE77AE086EE95E00E94DA2A2FC02E
:101DC00090E00E94740724E630E040E050E00E947A
:101DD000582ECA01B9012AE030E040E050E00E94EC
:101DE000582E49015A016B017C012AE030E0B5010F
:101DF000A40186EE95E00E94A32B6EE286EE95E0AC
:101E00000E94BE2A2AE030E0B701A60186EE95E0E6
:101E10000E94A32B63E786EE95E00E94FE2AFF90C6
:101E2000EF90DF90CF90BF90AF909F908F900895EC
:101E30001F93CF93DF9365E77AE086EE95E00E94EB
:101E4000982A8091A305813041F46CE57AE086EE12
:101E500095E00E94DA2A10E050C0823019F465E45F
:101E60007AE0F5CF843019F461E37AE0F0CF853081
:101E700091F766E27AE0EBCFC12FD0E0C930D1050F
:101E80000CF441C068E3610F86EE95E00E94BE2A23
:101E90006EE17AE086EE95E00E94982ABE016F5FBF
:101EA0007F4F4AE050E086EE95E00E94822B63E18E
:101EB0007AE086EE95E00E94982ACD55DA4FE981C6
:101EC000E03218F566E07AE086EE95E00E94982A06
:101ED0008981803130F06DE673E086EE95E00E94F6
:101EE000BB2A69816F7070E06F5F7F4F4AE050E0FE
:101EF00086EE95E00E948B2B1F5F80914C05181792
:101F000008F4BACF0FC061E3BECFEF70F0E0EE0F80
:101F1000FF1FEE56FC4F6081718186EE95E00E94B6
:101F2000EC2AEACF6BEE79E086EE95E00E94982AE3
:101F30008091BB050E94CF0E60ED79E086EE95E0C2
:101F40000E94982A8091BC050E94CF0E65EB79E033
:101F500086EE95E00E94982A8091BD050E94CF0EE2
:101F60006AE979E086EE95E00E94982A4091B305EF
:101F70005091B4056091B5057091B60541155105B4
:101F80006105710539F12AE030E086EE95E00E94A6
:101F9000C12B67E679E086EE95E00E94982A809151
:101FA000B7050E949907AB01BC012AE030E086EE3C
:101FB00095E00E94C12B63E479E086EE95E00E94F3
:101FC000982A4AE050E06091B80586EE95E00E94BC
:101FD000E92B06C06AE379E086EE95E00E94DA2AF2
:101FE0006DE179E086EE95E00E94982A6091B9054E
:101FF0007091BA054AE050E086EE95E00E94D32B3E
:1020000060E079E086EE95E00E94982A6091B20542
:10201000603450F470E06F5F7F4F4AE050E086EE2E
:1020200095E00E948B2B06C067EF78E086EE95E086
:102030000E94DA2A6AED78E086EE95E00E94982AFE
:102040008091B10580FF03C063EB71E002C067EBD4
:1020500071E086EE95E00E94EC2A6DEB78E086EE6A
:1020600095E00E94982A8091B10582700E94A50D8A
:102070006EE978E086EE95E00E94982A8091B1059D
:1020800084700E94A50D6FE778E086EE95E00E94CF
:10209000982A8091B10588700E94A50DDF91CF919B
:1020A0001F9108950F931F93CF93DF9320914905BC
:1020B0002F3FA9F56FEF75E086EE95E00E94982A14
:1020C00088E893E00E94730C6EED75E086EE95E073
:1020D0000E94982A80914A0590914B050E94730CAA
:1020E0006BEA75E086EE95E00E94DA2A68E875E012
:1020F00086EE95E00E94DA2A60E775E086EE95E0CC
:102100000E94DA2A6BE475E086EE95E00E94DA2AF6
:1021100086EE95E00E94C62A0E94180F68C012162B
:102120000CF065C0332727FD309580914C0590E079
:10213000821793070CF45BC066E375E086EE95E0CA
:102140000E94982A60914905772767FD70954AE0BB
:1021500050E086EE95E00E948B2B6BE075E086EEFA
:1021600095E00E94982A10E008E280914D0518172A
:10217000D0F5C12FD0E0CC0FDD1FC25BDA4F288134
:1021800030E080914905992787FD909501972817A0
:10219000390739F56BEB71E086EE95E00E94BB2ABA
:1021A0004AE050E0602F86EE95E00E94B22B6FEB84
:1021B00071E086EE95E00E94BB2AE981EF70F0E0C5
:1021C000EE0FFF1FEE56FC4F6081718186EE95E0A9
:1021D0000E94BB2A63EC71E086EE95E00E94BB2A68
:1021E0000F5F1F5FC2CF86EE95E00E94C62ADF9187
:1021F000CF911F910F910895FF920F931F93CF934B
:10220000DF93C9E8D5E0F12C8E0188818823D1F1D4
:1022100065EC71E086EE95E00E94BB2A4AE050E052
:102220006F2D86EE95E00E94B22B62ED71E086EE96
:1022300095E00E94BB2A2196F801208130E0A0E1C0
:10224000B7E20E94122E9B01AC01A0918805B0E07C
:102250000E94212EAB01BC0180917F0590918005E9
:10226000A0918105B0918205480F591F6A1F7B1FFD
:102270002AE030E086EE95E00E94C12BF394F8E16D
:10228000FF12C2CFCDB7DEB7E5E00C94C22E10929C
:10229000E30485E6E4EEF4E0DF011D928A95E9F7B8
:1022A0000895CF93C82F8F3719F0883009F045C0B3
:1022B000E091E304EE23D9F1E150E093E304F0E090
:1022C000EC51FB4F10826DE070E086EE95E00E94CD
:1022D0005906C0E08091E304C81760F4EC2FF0E0E9
:1022E000EC51FB4F608170E086EE95E00E9459064C
:1022F000CF5FF0CF60E270E086EE95E00E94590675
:102300006DE070E086EE95E00E945906C0E0809195
:10231000E304C81778F5EC2FF0E0EC51FB4F608137
:1023200070E086EE95E00E945906CF5FF0CF67E03F
:1023300086EE95E00E94BE2A1DC08B3119F40E94E2
:1023400047111AC08D30C1F08A30B1F08091E3049A
:10235000843668F76C2F70E086EE95E00E9459068F
:10236000E091E30481E08E0F8093E304F0E0EC5110
:10237000FB4FC08380E001C081E0CF910895CF93EF
:10238000C82F0E9400296093CC047093CD048093E1
:10239000CE049093CF04C093E104CC2329F040E015
:1023A00051EE60E070E004C040E855E260E070E0AB
:1023B00086EE95E00E94482DCF9108959091D0042B
:1023C000492F4F7050E0BA016F5F7F4F292F30E0E7
:1023D000E4E035952795EA95E1F76217730759F020
:1023E000FA01EF52FB4F808381E0890F8F70907F5D
:1023F000892B8093D00408956EE770E086EE95E017
:102400000E9459060895A3E1B1E0E9E0F2E10C94DD
:102410009C2EE9E8F5E0712C8191882321F07394DA
:1024200028E17212F9CF66ED71E086EE95E00E9428
:10243000EC2A4AE050E0672D86EE95E00E94E92BF9
:1024400080E00E94C10A0E949C0B8E010E5F1F4F0C
:10245000C12CD12C7601C39466246A945C2C0E9412
:10246000F4284B015C012091880530E0A0E1B7E23F
:102470000E94122E9B01AC01C701B6010E94342EAE
:1024800020917F0530918005409181055091820512
:10249000620F731F841F951F2091BF053091C005E7
:1024A0004091C1055091C2052617370748075907C3
:1024B00018F4F801608225C08C2D0E94F50961E0B6
:1024C00070E080E090E00E942329F80110820E94D1
:1024D000F428681979098A099B09643F71408105CC
:1024E000910540F40E940B0AF8019081981778F743
:1024F0008083EDCF50FE03C04298439A02C0429AB7
:1025000043982FEFC21AD20AE20AF20A0F5F1F4F56
:102510008FEFC816D104E104F10409F09FCFCE017A
:102520009395FC01D82E7FEF68EC2E2F281B2715E2
:1025300010F051E056C0DE01129651E02FEF41E05D
:102540003D91321710F0322F01C0452F5F5F5F3F82
:1025500011F0232FF5CF4193242F30E0A1E0B0E01C
:10256000AC0FBD1FA20FB31F5C93413079F0DE01A9
:10257000A20FB31F5C93423049F0AFEFBFEFAC0F37
:10258000BD1FA20FB31F6C934E3F78F6A2E0B0E0E0
:10259000AC0FBD1FA20FB31F7C934D3F30F6A3E0DD
:1025A000B0E0AC0FBD1FA20FB31F6C93BECF452F81
:1025B000242F30E0FC01E20FF31F6081AFEFB0E0A9
:1025C000AC0FBD1FA20FB31F2C91621748F44150EE
:1025D000DC01A40FB11D2C9120836C934111E8CF35
:1025E0005F5F571520F3372D369520E0231770F4E1
:1025F000DC01A20FB11D4C91522F530FFC01E50FCE
:10260000F11D50815C9340832E5FF0CFF9E8EF2EEF
:10261000F5E0FF2E8C01802F8D19871598F4F801B5
:10262000C1908F014AE050E06C2D86EE95E00E944B
:10263000B22B6CE286EE95E00E94BE2AF701C192B1
:102640007F01E9CF86EE95E00E94C62A81E0CD5E4B
:10265000DE4FEFE00C94B82E1F920F920FB60F9240
:1026600011241F932F933F934F935F936F937F9307
:102670008F939F93AF93BF93CF93DF93EF93FF938A
:10268000C0918600D0918700809187049091880442
:102690002091A904211155C09E01281B390B80915E
:1026A000C3059091C405A091C505B091C60585FDEF
:1026B00002C036952795253C49E03407B8F1409192
:1026C0000A0150E060E070E02CE1B695A79597957F
:1026D00087952A95D1F70097A105B10521F481E0EE
:1026E00090E0A0E0B0E084179507A607B707D8F4FC
:1026F00080910A018F3FB9F040E080910A014817AC
:1027000080F4842F90E0880F991FFC01E757FB4F5E
:1027100020813181FC01E55FFE4F318320834F5FD3
:10272000ECCF1092AA0410920A010BC02D3B82E05C
:10273000380720F080910A018031D8F08FEF809324
:102740000A01D0938804C0938704FF91EF91DF9131
:10275000CF91BF91AF919F918F917F916F915F9139
:102760004F913F912F911F910F900FBE0F901F908F
:10277000189510910A0181E0810F80930A01C90127
:102780000E942109E12FF0E0EE0FFF1FE757FB4FFA
:1027900091838083D6CF83E0809380008AE9809301
:1027A00081008091C30586FD05C080918100806411
:1027B000809381008FEF9FEF909389008093880032
:1027C00080916F00806280936F0008950E94710D68
:1027D0008091D805843011F41092D80508956F3097
:1027E00018F086958058089589E0689F802D1124FF
:1027F0000895A0E0B0E0EFEFF3E10C94A32EC82F12
:102800000E940029009138041091390420913A0463
:1028100030913B046B017C01C01AD10AE20AF30A31
:102820009701860149E8C41643E1D406E104F104A6
:1028300010F010923C046093380470933904809334
:102840003A0490933B042091A9048FEF820F8230C9
:10285000E8F5E0913C04EE2309F46EC1E13011F497
:1028600082E0D8C1E03178F581E08E0F80933C049E
:10287000F0E0E757FB4FC083803109F0D4C1EBE8AB
:10288000F4E0213029F4A181A695A695808108C0A5
:1028900080819181A92FA695A695A6959695879555
:1028A000A03148F4B0E090E0AA0FBB1FA55FBE4F77
:1028B00011969C938E931092AA04329684E0E93983
:1028C000F807F9F6B0C110923C04ADC1233009F00D
:1028D00023C1E0913C04E11118C0CF3009F011C1CF
:1028E0000E94F4280091B7041091B8042091B90413
:1028F0003091BA04601B710B820B930B623071052F
:102900008105910508F089C1FCC0E73148F481E0F8
:102910008E0F80933C04F0E0E857FB4FC083F1C07A
:10292000E73109F0ECC0C111EAC040E050E0ABE093
:10293000CA01B3E0880F991FBA95E1F7A49F9001EF
:10294000A59F300D1124F901E757FB4F6081E1810C
:102950007E2F777075956795FC01EE0FFF1FE55F81
:10296000FE4F71836083F901E657FB4FB081B69546
:10297000B695B695E181FE2FF295FF0FF07E6F2F91
:102980006B2BE695E695E6957E2F777075956795A6
:10299000FC01EE0FFF1FE35FFE4F71836083F901BF
:1029A000E557FB4FB081B295B695B695B370C1812E
:1029B000DC2FDD0FDD0F6D2F6B2BC295C695C695F5
:1029C000C370E281E170EE0FEE0F7E2F7C2B7595C8
:1029D0006795FC01EE0FFF1FE15FFE4F718360837F
:1029E000F901E357FB4FB081B695E181FE2FF795D2
:1029F000FF27F7956F2F6B2BE6957E2F77707595D8
:102A00006795FC01EE0FFF1FEF5EFE4F7183608341
:102A1000F901E257FB4FB081B295BF70E181FE2F03
:102A2000F295F07F6F2F6B2BE295EF707E2F777012
:102A300075956795FC01EE0FFF1FED5EFE4F7183EC
:102A40006083F901E157FB4FB081BB1FBB27BB1F60
:102A5000C181DC2FDD0F6D2F6B2BCC1FCC27CC1F42
:102A6000E281E370EE0F7E2F7C2B75956795FC015C
:102A7000EE0FFF1FEB5EFE4F71836083F901EF568F
:102A8000FB4FB081B695B695E181FE2FF295FF0F11
:102A9000FF0FF07C6F2F6B2BE695E6957E2F7770FE
:102AA00075956795FC01EE0FFF1FE95EFE4F718380
:102AB0006083F901EE56FB4F208122952695277001
:102AC0003181E32FEE0FEE0FEE0F6E2F622B732F7F
:102AD00072957695777075956795FC01EE0FFF1FDF
:102AE000E75EFE4F718360834F5F5F4F4230510559
:102AF00009F01ECF80919F0483FF1092AA041092C8
:102B00003C040E94F4286093B7047093B804809347
:102B1000B9049093BA0487C0243009F084C060914E
:102B20003C0461110BC0C83AB1F4109279051092BF
:102B3000780588EA0E94610681E06CC0613019F472
:102B4000C093370404C0623031F4C09336048C2F34
:102B50000E9461065AC0E09136042E2F30E0220F09
:102B6000331F462F50E0C9010296841795073CF0A9
:102B7000633268F7FA01EA57FB4FC083E8CF2D5F55
:102B80003F4F8C2F90E06091780570917905421746
:102B9000530749F4982F882786279727909379051C
:102BA0008093780532C06817790769F580913704FA
:102BB000813049F5E13118F080E180933604F090DE
:102BC0003604CAE8D4E000E010E00F15D0F4FE01AE
:102BD0003197808190E0982F88272881822B63E0AD
:102BE000969587956A95E1F70E942109F801EE0F05
:102BF000FF1FE55FFE4F918380830F5F1F4F22967B
:102C0000E4CF1092AA0410923C0480913C048823E3
:102C100051F08F5F80933C0406C080913C048F5F2D
:102C200080933C046ECFCDB7DEB7E8E00C94BF2EA6
:102C3000E82FF0E0E254FA4FE185E03150F4F894E7
:102C4000F0E0EE0FFF1FE55FFE4F808191817894E9
:102C500008958EE08E0F8B3058F4F0E0E25FF109BA
:102C600024E62E9FC0012F9F900D11240C960895ED
:102C7000E03FF1F028F4E03161F0E13161F006C0AD
:102C8000ED3F81F0EE3F89F0E13F49F080E092E0D6
:102C9000089582E101C083E10E94422A089586E0FE
:102CA00090E008958AEF93E008958FEF93E0089500
:102CB00080E090E00895A2E2B0E0E1E6F6E10C9455
:102CC000992E9E012F5F3F4F80E1D9011D928A9579
:102CD000E9F764E072E086EE95E029A33AA30E944A
:102CE000EC2A0E94BF0B1D8A1E8A1F8A188E312C67
:102CF000212C00E0812C912C5401412C74E7572E9B
:102D00007BE8672E72E3772EE0E5CE2EE3ECDE2E35
:102D1000E12CF12C84EF91E0A0E0B0E08D8F9E8F4C
:102D2000AF8FB8A380E09EECADEEB4E3898F9A8FAD
:102D3000AB8FBC8F80E094E7ABE8B2E3898B9A8BD2
:102D4000AB8BBC8B86EE95E00E94002C892B09F49E
:102D5000E1C086EE95E00E942D2C9C0133272C3299
:102D6000310509F442C0ACF42332310509F0ABC09F
:102D700019821A821B821C821D821E821F82188663
:102D800019861A861B861C861D861E861F86188A33
:102D900060C02434310529F02335310509F4B2C06F
:102DA00092C064E486EE95E00E94BE2A2AE030E0FC
:102DB00040E054E76BE872E386EE95E00E944C2B0E
:102DC0006CE286EE95E00E94BE2A2AE030E040E008
:102DD0005EEC6DEE74E386EE95E00E944C2B6CE2A7
:102DE00086EE95E00E94FE2AADCF0F5F043009F019
:102DF000A9CF29813A814B815C81A8EEB3E00E9482
:102E0000212E698B7A8B8B8B9C8B2D813E814F8100
:102E100058850E94212E698F7A8F8B8F9C8F2985F0
:102E20003A854B855C852D8F3E8F4F8F58A32D851E
:102E30003E854F8558890E94212E6B017C016032AE
:102E40003EE473078105910530F462E38CE10E9452
:102E5000E20900E077CF603345E77407810591050B
:102E600010F462E2F3CF60345CE9750781059105E7
:102E700010F466E2EBCF80E5C81683ECD806E104D7
:102E8000F10410F462E1E2CF90E6C9169AEED90699
:102E9000E104F10410F465E1D9CFA0E7CA16A1E17D
:102EA000DA06A1E0EA06F10410F461E0CFCFB0EA5F
:102EB000CB16B6E8DB06B1E0EB06F10410F463E0F4
:102EC000C5CF65E0C3CF10ED180F1A3008F03ACF28
:102ED000E1E0F0E0EC0FFD1F24E0029FE00DF11DAA
:102EE00011242081318142815381AAE0B0E00E9407
:102EF000212E610F711D811D911D6083718382835D
:102F0000938320CF49885A886B887C88812C912CA8
:102F1000540118CF81149104A104B10489F4C301B0
:102F2000B2010E94510A61E070E080E090E00E94EE
:102F300023291D8A1E8A1F8A188E312C22242A9446
:102F40008D8D9E8DAF8DB8A188169906AA06BB06F9
:102F5000D0F40E940B0A2D893E894F89588D280F85
:102F6000311D411D511D2D8B3E8B4F8B588F3816B7
:102F700008F4382E821508F4282E3FEF831A930A9E
:102F8000A30AB30A56C0C301B20128EE33E040E001
:102F900050E00E94582EBA01A9012AE030E086EEE6
:102FA00095E00E94A32B6CE286EE95E00E94BE2A7B
:102FB0004AE050E0632D86EE95E00E94B22B6CE271
:102FC00086EE95E00E94BE2A6D897E898F89988D54
:102FD000A50194010E94582EBA01A9012AE030E00F
:102FE00086EE95E00E94A32B6CE286EE95E00E94AF
:102FF000BE2A4AE050E0622D86EE95E00E94B22B98
:103000006CE286EE95E00E94FE2A4C0C5D1C6E1C64
:103010007F1C898D9A8DAB8DBC8D84159505A60579
:10302000B70520F449885A886B887C88812C912CBC
:10303000540129893A894B895C89283E33404105EE
:10304000510509F07FCEA296E2E10C94B52EACE1D9
:10305000B0E0EDE2F8E10C94A32E0E9400296B0190
:103060007C0181E00E94C10A14E703E0198361E05A
:10307000CE0101960E941E0C009377050E949C0BC6
:103080006AEF70E080E090E00E942329809177054C
:10309000833089F486EE95E00E94002C892B59F448
:1030A0000E9400296C197D098E099F096038734CB4
:1030B000894C9140D8F280917705833009F44FC054
:1030C0008FE70E94BA090E94CD098983843511F0E7
:1030D00083E05CC00E94CD0910924A0580934B05A5
:1030E0000E94CD0920914A0530914B05280F311DD2
:1030F00030934B0520934A050E94CD0980934C05DF
:103100000E94CD0980934D05813110F7F12C0F2DD0
:1031100010E080914D0590E0880F991F081719075E
:1031200040F40E94CD09F801E25BFA4F8083F394EA
:10313000EECF80E7898361E0CE0101960E941E0CEC
:1031400083E0809377050E949C0B62E370E080E04F
:1031500090E00E94232980917705833011F482E06A
:1031600015C08FE70E94BA090E94CD098983803576
:1031700009F0AECF03EA15E00E94CD09F801819372
:103180008F01F5E00E3B1F07B9F781E06C96E8E090
:103190000C94BF2E80914905992787FD9095A92F02
:1031A000B92FFC013196EB30F10508F066C0EC5CFC
:1031B000FF4F0C94D02E62E778E086EE95E00E94F7
:1031C000DA2A88E893E00E94730C6AE578E086EEDC
:1031D00095E00E94DA2A65E378E086EE95E00E94A9
:1031E000DA2A6BE078E086EE95E00E94DA2A6AEE51
:1031F00077E086EE95E00E94DA2A6DEB77E086EEC6
:1032000095E00E94DA2A67E977E086EE95E00E9471
:10321000DA2A63E777E086EE95E00E94DA2A6CE42A
:1032200077E086EE95E00E94DA2A86EE95E00E942D
:10323000C62A0E94B10D21C06FE277E01AC06AE091
:1032400077E017C065EF76E014C066ED76E011C058
:1032500062E976E00EC06DE776E00BC068E676E0E6
:1032600086EE95E00E94DA2A62E276E002C06CE027
:1032700076E086EE95E00E94DA2A6AE070E080E06F
:1032800090E00E94232986EE95E00E94002C892B75
:1032900029F086EE95E00E942D2CF5CF0895ACE143
:1032A000B0E0E5E5F9E10C94A32E909149059F3F2C
:1032B00009F023C1482F50E0FA013A97EF36F105A3
:1032C00008F00FC1E15CFF4F0C94D02E61E172E079
:1032D000A0C06DE172E086EE95E00E94EC2A85E7E1
:1032E00089838BE1E3EAF5E0DE01129601900D920D
:1032F0008A95E1F76CE1CE0101960E941E0C0E94B6
:103300009C0B83E08093770568EC70E080E090E0B0
:103310000E94232980917705843009F0E2C08FE76D
:103320000E94BA090E94CD098983853509F0D9C068
:103330006DEE74E086EE95E00E94DA2A6FEC74E0A0
:1033400086EE95E00E94DA2A61EB74E096C065E3B0
:1033500072E086EE95E00E94EC2A89E6898361E0BE
:10336000CE0101960E941E0C0E949C0B83E080936C
:10337000770568EC70E080E090E00E94232980915E
:103380007705843009F0ADC08FE70E94BA090E942A
:10339000CD0989838E010E5F1F4F7E014DE1E40E42
:1033A000F11C0E94CD09F80181938F01EE15FF05F4
:1033B000C1F78BE1FE013296A3EAB5E001900D92D0
:1033C0008A95E1F78981893409F08BC063E974E05B
:1033D00086EE95E00E94DA2A65E774E086EE95E0D5
:1033E0000E94DA2A67E574E048C06FE472E086EE76
:1033F00095E00E94EC2A8EEF8093490572C08052BE
:103400008750805390914C05981708F066C06EE580
:1034100072E086EE95E00E94EC2A63C084E180931E
:10342000490560E274E029C085E18093490569EEB1
:1034300073E023C086E18093490562EB73E01DC011
:1034400087E18093490568E673E017C088E18093BF
:10345000490567E573E011C089E18093490563E49C
:1034600073E00BC08AE1809349056EE273E005C00A
:103470008BE18093490566E073E086EE95E00E945B
:10348000DA2A2FC06CEE72E086EE95E00E94DA2A0E
:103490008091B10591E01DC066ED72E086EE95E089
:1034A0000E94DA2A8091B10592E013C061EC72E0CB
:1034B00086EE95E00E94DA2A8091B10594E009C079
:1034C00066EA72E086EE95E00E94DA2A8091B10504
:1034D00098E089278093B1058FEF809349050E947A
:1034E000521086EE95E00E94002C892B09F45AC1F7
:1034F00086EE95E00E942D2CF4CF0E945111882376
:1035000009F450C18091E304811104C08FEF8093CE
:10351000490540C140E050E060E070E084EE94E096
:103520000E94472F40914905042F112707FD109550
:10353000212F312FF8013197EB31F10508F01AC135
:10354000E255FF4F0C94D02E552747FD5095209102
:103550004C0530E0241735070CF40CC18B019C019D
:1035600001501109210931090032110521053105E8
:1035700058F0C0904D05EFE4F5E0F12CD12CA8E215
:10358000EA2E415051090FC0FA01ED55FA4F615032
:103590006083D8C0DF0111972C9130E024173507E4
:1035A00029F0F3943296FC10F5CFCAC00E2D10E02E
:1035B00020E030E0061717072807390741F420817B
:1035C000DA01AD55BA4F11962C93DD24D394E394D0
:1035D000E8CF6F3F71058105910511F008F0CAC071
:1035E0006093BB05AFC06F3F71058105910511F078
:1035F00008F0C0C06093BC05A5C06F3F7105810590
:10360000910511F008F0B6C06093BD059BC02091F4
:10361000E40420622037E9F440E050E060E070E02C
:1036200085EE94E00E94472F9B01AC01DC01CB01A9
:103630000197A109B1090897A105B10508F0ADC02E
:10364000A4EDB0E30E94212E6A5E7C4A8A46954E24
:1036500024C02636E9F440E050E060E070E085EEFA
:1036600094E00E94472F9B01AC01DC01CB01019744
:10367000A109B1090797A105B10508F08EC0A8EA14
:10368000B1E60E94212E645E7C438E46944E05C0B6
:10369000611571058105910571F08B019C0114572D
:1036A0002B4832430130FAE51F07F2E62F07F2E01C
:1036B0003F0708F05FC06093B3057093B405809333
:1036C000B5059093B6053EC06F3F71058105910524
:1036D00011F008F04FC06093B70534C08B019C0116
:1036E00001501109210931090F3F1105210531054B
:1036F00008F040C06093B80525C08B019C01045CB4
:103700001940210931090D344DE114072105310516
:1037100028F47093BA056093B90514C0611571055A
:103720008105910521F48FEF8093B2050BC06134C0
:10373000710581059105F0F461506093B20502C0F6
:10374000DD20C1F08091E20481111AC080918305CF
:1037500090918405A0918505B09186050196A11DE3
:10376000B11D8093830590938405A0938505B09344
:10377000860506C060E772E086EE95E00E94EC2ABE
:103780000E9447118FEF809349056AE086EE95E02D
:103790000E94FE2A0E94521005C061E070E080E0A5
:1037A00090E07BCF6C96E8E00C94BF2E6AE572E067
:1037B00086EE95E00E94DA2A62E472E086EE95E0F9
:1037C0000E94DA2A86EE95E00E94002C892B31F0C7
:1037D00086EE95E00E942D2C0E944F190E9427181A
:1037E000823029F0833051F46DE072E002C064E26F
:1037F00072E086EE95E00E94DA2A08958FEF8093BA
:1038000049051092E2040E945210809149058E3FB2
:1038100069F086EE95E00E94002C892BB1F386EECC
:1038200095E00E942D2C0E944F19EFCF08950F9321
:103830001F93109149051F3F09F0D2C0893409F444
:1038400057C000F5883309F469C058F4803309F48F
:1038500077C008F061C08B3109F440C08132B1F10A
:10386000B9C0813409F487C030F4893309F466C0E3
:10387000803461F1AFC0823409F48EC0863409F41B
:1038800048C0A8C0823609F487C078F4883531F181
:1038900028F48235C1F18335E1F09CC08A3509F402
:1038A00094C0813609F467C095C0823761F128F46D
:1038B000863679F18936E1F08DC0883779F08A371C
:1038C00009F483C0833709F085C003C061E172E069
:1038D00015C00E94820D6EE872E004C00E948B0D3C
:1038E00068EA72E086EE95E00E94EC2A8EEF70C0E6
:1038F0000E947A060E94BF0667EC72E086EE95E0B1
:103900000E94EC2A67C081E00E94DF0660EE72E050
:10391000F5CF0E94FC105EC080535AC06AEF71E080
:1039200086EE95E00E94DA2A9091A20588E0890F40
:103930008871977E892B8093A2051AC089E048C0C0
:1039400067EE71E086EE95E00E94DA2A8091C30569
:103950009091C405A091C505B091C60520E18227CC
:103960008093C3059093C405A093C505B093C60585
:10397000109349052FC061ED71E086EE95E00E943D
:10398000DA2A8091C3059091C405A091C505B09134
:10399000C60540E4842710C060EC71E086EE95E037
:1039A0000E94DA2A8091C3059091C405A091C505B3
:1039B000B091C60520E282278093C3059093C40589
:1039C000A093C505B093C60502C00E94D61B8FEF19
:1039D00080934905809149058E3F09F0D4C0DDC030
:1039E0000E945111882309F4D8C08091E304811109
:1039F00004C08FEF80934905C6C040E050E060E00E
:103A000070E084EE94E00E94472F00914905112751
:103A100007FD1095212F312FF8013197E930F1057D
:103A200008F0B4C0E753FF4F0C94D02E8B019C01DB
:103A3000015014472B4832430F3F1945224632406C
:103A400008F0A4C060937F05709380058093810582
:103A50009093820577C0609383057093840580936B
:103A600085059093860581E08093E2046BC0683001
:103A700071058105910508F089C06093870562C0D2
:103A80008B019C0101501109210931090A301105EE
:103A90002105310508F07AC06093880553C061EBB9
:103AA00071E084EE94E00E94813010E0009799F07C
:103AB0000E945B30009779F0183130F4E12FF0E08C
:103AC000E658FA4F87871F5F61EB71E080E090E076
:103AD0000E948130EBCF1831A8F5E12FF0E0E658D5
:103AE000FA4F17861F5FF7CF653071058105910585
:103AF00008F04CC06093A10525C08B019C010150CA
:103B00001109210931090630110521053105F0F5AA
:103B10002091A205287F262B2093A20513C08B019C
:103B20009C0101501109210931090115124C214054
:103B3000310560F560937B0570937C0580937D056E
:103B400090937E058091E204811113C080918305DA
:103B500090918405A0918505B09186050196A11DDF
:103B6000B11D8093830590938405A0938505B09340
:103B700086050E9447118FEF809349056AE086EE23
:103B800095E00E94FE2A0E94CA1807C060E772E012
:103B900086EE95E00E94EC2AECCF1F910F910895DC
:103BA0008FEF809349051092E2040E94CA18809119
:103BB00049058E3F69F086EE95E00E94002C892B26
:103BC000B1F386EE95E00E942D2C0E94171CEFCFDA
:103BD0006AE070E080E090E00E94232986EE95E0A4
:103BE0000E94002C892B29F086EE95E00E942D2C56
:103BF000F5CF0895CF93C82F682F86EE95E00E94E9
:103C00005A2C90916E059C2790936E05CF91089544
:103C1000A1E0B0E0EEE0FEE10C94A92E99830E94B1
:103C2000FA1D9981892F0E94FA1D2196E2E00C94D9
:103C3000C52E1F93CF93DF93182FEB0110926E05C3
:103C400065EB70E086EE95E00E94590662E670E052
:103C500086EE95E00E945906812F0E94FA1DCE0142
:103C60000E94081EDF91CF911F91089560916E050B
:103C700086EE95E00E945A2C0895A1E2B0E0E3E4BC
:103C8000FEE10C94A52E7B018A018C3009F453C10E
:103C900008F040C0863009F4BCC018F5833009F440
:103CA00091C070F4813009F472C0823009F04AC2C8
:103CB0006BE170E082E00E94191E03EA15E078C013
:103CC000843009F487C0853009F03CC260914D050D
:103CD00070E0660F771F85E00E94191E0EE415E064
:103CE00086C0893009F4A7C070F4873009F49BC0FE
:103CF000883009F027C261E070E088E00E94191E58
:103D00008091D80525C28A3009F4CAC08B3009F4E5
:103D1000F2C018C28A3609F475C1D8F4873609F49E
:103D20003AC138F4853609F40EC1863609F41FC14C
:103D300009C2883609F437C1893609F003C261E047
:103D400070E089E60E94191E0E947A060E94BF0652
:103D5000F7C18D3609F4D4C138F48B3609F491C11A
:103D60008C3609F49AC1EEC18E3609F4DEC1873C67
:103D700009F0E8C161E070E087EC0E94191E81E063
:103D80000E94FA1D0E94361E10926F05E5C169E27D
:103D900070E081E00E94191E0AE715E0F8018191A8
:103DA0008F010E94FA1DF5E0033A1F07B9F7D2C14F
:103DB000F80181918F010E94FA1DF5E00E3B1F076B
:103DC000B9F7C8C161E070E083E00E94191E0E944B
:103DD0002718BEC161E070E084E00E94191E81E0F6
:103DE0000E94FA1D0E94361E0E945B16B5C180918A
:103DF0004D0590E0880F991F98012E5435402817E3
:103E0000390708F0A7C1F80181918F010E94FA1DBE
:103E1000EECF62E070E086E00E94191E88E893E031
:103E20000E94081E97C161E070E087E00E94191EA1
:103E300080914C058DC186E6898361E0CE010196B3
:103E40000E941E0C0E949C0B83E08093770568EC17
:103E500070E080E090E00E94232980917705843013
:103E6000D9F48FE70E94BA090E94CD09898386346C
:103E700069F460E270E089E00E94191E10E20E947D
:103E8000CD090E94FA1D1150D1F764C161E070E0C4
:103E900089E00E94191E54C161E070E089E055C1BB
:103EA00069E170E08AE00E94191E81E08093BE05FE
:103EB000209176058091C3059091C405A091C50518
:103EC000B091C605222311F0806801C08F778093DE
:103ED000C3059093C405A093C505B093C6050EEB2A
:103EE00015E0F80181918F010E94FA1DF5E0073D70
:103EF0001F07B9F72FC161E270E08BE00E94191E25
:103F00008091AA048F3F39F08091AA0491E0980F24
:103F10009093AA0402C08091AA040E94FA1D10E0A6
:103F2000812F0E9418160E944C090E94081E1F5FD4
:103F30001031B1F70FC161E070E08CE00E94191EF2
:103F40008091D70505C161E070E085E60E94191EE9
:103F500089E2E816F10409F0FAC0D801EAE7F5E0D1
:103F60008D91819385E0E33AF807D1F7E9C061E0EC
:103F700070E086E60E94191EEBE1EE16F10409F0EE
:103F8000E6C0D801E3EAF5E08D91819385E0EE3B50
:103F9000F807D1F7D5C061E070E087E60E94191EEE
:103FA0000E94820DCDC061E070E088E60E94191E7B
:103FB00085E789838BE1E3EAF5E0DE011296019063
:103FC0000D928A95E1F76CE1CE0101960E941E0CDC
:103FD0000E949C0B83E08093770560E273E080E0B1
:103FE00090E00E94232980917705843009F0AFC0CA
:103FF0008FE70E94BA090E94CD098983853509F0AF
:10400000A6C09EC061E070E08AE60E94191E89E6A3
:10401000898361E0CE0101960E941E0C0E949C0BD8
:1040200083E08093770560E273E080E090E00E9497
:10403000232980917705843009F089C08FE70E9499
:10404000BA090E94CD0989838E010E5F1F4F7E0140
:10405000EDE1EE0EF11C0E94CD09F80181938F0174
:10406000EE15FF05C1F78BE1FE013296A3EAB5E03C
:1040700001900D928A95E1F78981893409F067C032
:104080005FC061E070E08BE60E94191EF80180813C
:104090008093D8050E948B0D53C061E070E08CE6E0
:1040A0000E94191EF0E2EF16F10461F487E689839D
:1040B00080E2F801DE01129601900D928A95E1F7F7
:1040C00061E203C087E4898361E0CE0101960E942A
:1040D0001E0C0E949C0B83E0809377056CE474E0D7
:1040E00080E090E00E94232980917705843079F563
:1040F0008FE70E94BA090E94CD09873441F520C09C
:1041000061E070E08DE60E94191E89E1E816F10475
:10411000F1F4D801EEEBF5E08D91819385E0E73D78
:10412000F807D1F70E94CB130BC061E070E08EE678
:104130000E94191EF80180818093D7050E946C0DA2
:1041400081E006C061E070E08AEC0E94191E80E008
:104150000E94FA1D0E94361EA196E6E00C94C12E24
:10416000A0E0B0E0E6EBF0E20C94A32ECAECD3E0C2
:1041700014E606E035E0F32E44E0E42E53E0D52EBD
:1041800062E0C62E86EE95E00E94002C892B09F491
:104190009BC086EE95E00E942D2C282F809335043D
:1041A0004091340450E04730510560F7FA01EE5277
:1041B000FF4F0C94D02E853B29F781E08093340487
:1041C000E1CF823609F07DC0C0923404DBCF80930A
:1041D000330480933204D0923404D4CF9C0133272B
:1041E00030933104209330049091320498279093B7
:1041F0003204E0923404C6CF382F22274091300495
:1042000050913104242B352B30933104209330040A
:1042100090913204982790933204F092340425361A
:10422000310508F4AFCF61E070E08CEC0E94191EFC
:1042300081E00E94FA1D0E94361E43C020912E0488
:1042400030912F04F901E653FC4F808390913204A2
:10425000982790933204C901019690932F0480937C
:104260002E0420913004309131048217930708F412
:1042700089CF0093340486CF8091320482130BC01F
:1042800060912E0470912F044AEC53E08091330426
:104290000E943D1E0DC062E070E08BEC0E94191E72
:1042A000809133040E94FA1D80916E050E94FA1DD0
:1042B000FE01812F11928A95E9F710922F04109236
:1042C0002E04109234045ECFCDB7DEB7E8E00C9434
:1042D000BF2E81E080936F0580916F05882349F0A0
:1042E00086EE95E00E94002C892BB1F30E94B0204D
:1042F000F3CF0895AAE2B0E0E0E8F1E20C94A12E39
:104300000E94F4286B017C0181E00E94C10A86EEC4
:1043100095E00E94002C892B29F086EE95E00E9402
:104320002D2CF5CF439811E072E6B72EE9E2AE2EC0
:1043300003E00E94F4286C197D098E099F09693CED
:10434000710581059105D0F11123C1F10E94F42876
:104350006B017C01429A80ED97E00E94B607B9821A
:10436000EAE7F5E0DE0112968A2D01900D928A951A
:10437000E1F76AE2CE0101960E941E0C429880E0AD
:1043800090E00E94B607009377050E949C0B62E3C1
:1043900070E080E090E00E942329809177058430CE
:1043A00061F4009377058FE70E94BA090E94CD0956
:1043B00011E0823419F410E001C011E082E10E94A2
:1043C000192A892B81F411E00EC0439A429A86EE95
:1043D00095E00E942D2C8D309105A9F05CF40A9790
:1043E00091F04398429886EE95E00E94002C892B2C
:1043F00061F79FCF8332910579F08234910589F777
:104400000E946921EECF62EB71E086EE95E00E949A
:10441000DA2A0E94D01DE5CF0E945B16E2CF8F9270
:104420009F92AF92BF92CF92DF92EF92FF921F9333
:10443000CF93DF9382E10E94192A892B09F089C06A
:1044400068EC70E080E090E00E94232980E090E03A
:104450000E94B6070E94F4284B015C016B017C01AD
:1044600080ECC80E82E1D81EE11CF11C0E94F428E9
:104470006C157D058E059F0530F482E10E94192A96
:10448000892BA1F364C082E10E94192A892B09F0CB
:104490005EC080ED97E00E94B6070E94F4286B0191
:1044A0007C01D0E0C1E088E4880E86E2981EA11C61
:1044B000B11C11E082E10E94192A892B21F58C148C
:1044C0009D04AE04BF0430F480ED97E00E94B6076F
:1044D000D1E0F0CF0E94F4286C197D098E099F0964
:1044E000693C71058105910528F30E94F4286B0150
:1044F0007C01C12719F080ED97E002C080E090E0D8
:104500000E94B607D7CF80E090E00E94B607DD2377
:10451000B9F08091D70590E0019665E070E00E94C7
:10452000442E8093D7050E946C0D0E94E6130E94D2
:104530008B0D64EF71E080E090E00E94232909C0B8
:1045400080E00E94DF060E9403120E94820D0E94FA
:104550007A21DF91CF911F91FF90EF90DF90CF9064
:10456000BF90AF909F908F900895CF92DF92EF927F
:10457000FF9280E00E941D080E94F40761E081E143
:104580000E94AD2961E080E10E94AD2960E082E1F6
:104590000E94AD2960E088E00E94AD2961E088E0DA
:1045A0000E94E6290E949F0740E052EC61E070E023
:1045B00086EE95E00E94482D0E94E6130E948B0D26
:1045C0000E94CB138FEF8093AA040E94090878946D
:1045D0000E94F4286B017C018091AA048F3F59F45A
:1045E0000E94F4286C197D098E099F09603D77406F
:1045F0008105910588F380ED97E00E94B60761E0A0
:1046000082E10E94E629439A86EE95E00E94002C02
:10461000892B29F086EE95E00E942D2CF5CF6DEFC9
:1046200072E086EE95E00E94BB2A88E893E00E9443
:10463000730C64E173E086EE95E00E94BB2A4AE0C9
:1046400050E068E070E086EE95E00E948B2B62E31C
:1046500070E080E090E00E94232986EE95E00E94C1
:10466000002C04970CF186EE95E00E942D2C8234EC
:104670009105D1F486EE95E00E942D2C8E349105A3
:1046800099F486EE95E00E942D2C8434910561F416
:1046900086EE95E00E942D2C819731F480E090E029
:1046A0000E94B6070E947A2140917B0550917C05BB
:1046B00060917D0570917E05DB01CA010197A1091A
:1046C000B1090497A105B10568F44093A9044330EA
:1046D00029F440EA56E861E070E004C040E052ECA2
:1046E00061E070E086EE95E00E94482D0E940F2266
:1046F000439880E090E00E94B6070E94CB1310928E
:10470000C9048091C30583FF11C080918F05882360
:1047100051F080919605882331F080919D05882382
:1047200011F087E001C085E08093C90480E00E9419
:10473000C10A8091CA040E94F5090E949C0B109244
:104740003F0410923E0410923D04F12C8091D80554
:104750008F15B0F062E370E080E090E00E942329C2
:1047600080ED97E00E94B60762E370E080E090E0A1
:104770000E94232980E090E00E94B607F394E6CFE0
:104780008091A20584FF08C0982F987181E098312C
:1047900009F080E00E94BF118FE00E941D08FF9089
:1047A000EF90DF90CF900895EF92FF920F931F93B9
:1047B000CF93DF938C016EE770E086EE95E00E9468
:1047C0005906E801F12CF0E2EF2E8E0188818D5719
:1047D000823048F46DE770E086EE95E00E9459065D
:1047E00088818E2588832196F801608186EE95E088
:1047F0000E945A2CF394F9E0FF12E7CF6EE770E0C5
:1048000086EE95E00E945906CDB7DEB7E6E00C943F
:10481000C12EA9E0B0E0EFE0F4E20C94A92E909153
:10482000CB0491110EC09EEF99838A836B8350E075
:10483000559547954C832D83198618861F821E82B5
:104840002EC04091D004842F90E0B4E095958795D8
:10485000BA95E1F7242F2F7030E08217930719F1F2
:104860008DEF89831B82FE01349650E0842F90E007
:10487000A4E095958795AA95E1F7242F2F7030E055
:104880008217930749F0DC01AF52BB4F8C918193A3
:10489000405F5F5F563051F74093D0045A83CE019A
:1048A00001960E94D4238091CB0490E0019666E0AB
:1048B00070E00E94442E8093CB042996E2E00C9491
:1048C000C52EA0E0B0E0E7E6F4E20C94A22E6C0165
:1048D0006EE770E086EE95E00E9459068601E12CB5
:1048E000F12CC0E0D0E030E2B32EF801608183E823
:1048F000860F823078F46DE770E086EE95E00E94D6
:104900005906F80160816B2570E086EE95E00E9403
:10491000590604C086EE95E00E945A2CE114F10479
:1049200059F0F80180819E01280F311DC901C92F5E
:10493000DD27C80FD91FDD273FEFE31AF30A89E00F
:10494000E816F10459F028E0E216F10421F48C2F66
:104950008095F60180870F5F1F4FC7CFCDB7DEB7B9
:10496000E9E00C94BE2EA9E0B0E0E9EBF4E20C948F
:10497000A92EE82F362F8091CB0490E0019664E2B7
:1049800070E00E94442E8093CB0458E9598350E193
:104990005A83813089F048F08230B9F08330D9F4FD
:1049A0008B8381EF8C833D8319C085E08B8381EFFE
:1049B0008C832F5F2D8312C08B8381EF8C8384E6E1
:1049C000489FA00111245D8309C084E08B8381EF9F
:1049D0008C83ED8303C00E94FC1104C0CE010196BC
:1049E0000E9461242996E2E00C94C52EA2E0B0E07A
:1049F000ECEFF4E20C949E2E182F762E2A83498336
:104A00000E9400296B017C018091E1048090CC041C
:104A10009090CD04A090CE04B090CF042A8149811B
:104A20008823C1F0D701C60188199909AA09BB09D1
:104A30004C015D0191EE89169EE29906A104B10434
:104A400020F1241708F4422F202F672D812F0E9478
:104A5000B32413C0D701C60188199909AA09BB0953
:104A60004C015D0191E3891695E79906A104B10413
:104A700060F0672D812F0E940924C092CC04D0924F
:104A8000CD04E092CE04F092CF042296EDE00C9497
:104A9000BA2EA2E2B0E0EFE4F5E20C949F2E8CE097
:104AA0000E94DC0981110DC06CE173E086EE95E097
:104AB0000E94EC2A439A80E00E94C10A0E949C0B4B
:104AC000439886EE95E00E94002C892B01F186EE3A
:104AD00095E00E942D2C9091A904992319F00E9431
:104AE000F913EFCF40913E0450E09A012F5F3F4F02
:104AF0002F71332760913F0470E02617370709F3C1
:104B0000FA01E75BFB4F808320933E04DACF80916C
:104B10007705843009F086C00E940029611571056F
:104B20008105910549F06093BB047093BC048093A8
:104B3000BD049093BE040CC081E090E0A0E0B0E022
:104B40008093BB049093BC04A093BD04B093BE04B7
:104B50008091AD049091AE0481609093AE048093F7
:104B6000AD0483E0809377058FE70E94BA0909E6D8
:104B700014E00E94CD09F80181938F01F4E002371F
:104B80001F07B9F72091720480916904982F92272A
:104B900096FF3BC090E4922790937204982F9873ED
:104BA0009833F1F410E0212F30E080916904877090
:104BB00090E0821793074CF11F5F2091A205812F8F
:104BC00090E0FC01E759FB4F24FF04C080810E9464
:104BD000DE11E9CF608186EE95E00E945A2CE3CF8A
:104BE0008F7399F480916A048093B60480916B046A
:104BF0008093B40480916C048093B30480916F041B
:104C000090E09093AC048093AB0480913D0481309C
:104C100019F482E080933D0480913D04833011F4C7
:104C200010923D040E9400296B017C018091AF0429
:104C30009091B004A091B104B091B2040097A10585
:104C4000B105C9F0A7019601281B390B4A0B5B0B74
:104C5000DA01C901883B9B40A105B10560F00E94C3
:104C60000B0A8093B5041092AF041092B004109216
:104C7000B1041092B2048091BF049091C004A0913D
:104C8000C104B091C20446015701881A990AAA0AC0
:104C9000BB0A8AE795E00E94370886169706A806A1
:104CA000B90608F4A8C0C092BF04D092C004E09234
:104CB000C104F092C2040E9457068091AA04883071
:104CC000A0F08091C3059091C405A091C505B09155
:104CD000C6055CE1B695A795979587955A95D1F746
:104CE000892B8A2B8B2B09F0AAC18091AA048F5F94
:104CF0008093AA048091BB049091BC04A091BD0450
:104D0000B091BE040097A105B105F1F0C81AD90A07
:104D1000EA0AFB0A8AE795E00E9437086C157D05D0
:104D20008E059F0508F012C18091C30584FD04C063
:104D300080ED97E00E94B6071092BB041092BC046D
:104D40001092BD041092BE0490917204907C9093D6
:104D5000720450913E0480913F0420913D04581705
:104D600009F411C1223009F00EC1905890937204D9
:104D7000E091A205E770F0E0E658FC4F60816930F1
:104D800008F0E9C0615040E04613E7C080933F045B
:104D900087E3840F90917204892B8093720440936F
:104DA000400483E080933D04429A8091870590916E
:104DB000C904911135C10E94BC0A8091CA040E94A5
:104DC000F509E091A205E770F0E0E658FC4F60813C
:104DD00082E794E00E94D70BE091CA04EF5FE09372
:104DE000CA04E83109F428C1F0E0E658FA4F878593
:104DF000882309F421C10E94460C813069F5809115
:104E0000A205887149F18091AD049091AE04880F9C
:104E1000991F9093AE048093AD0483E0809377054F
:104E20000E949C0B0E9400296093AF047093B00411
:104E30008093B1049093B204672B682B692B61F4C3
:104E400081E090E0A0E0B0E08093AF049093B004E4
:104E5000A093B104B093B2048091A20584FF2BC04B
:104E60008091BB049091BC04A091BD04B091BE049C
:104E7000892B8A2B8B2BF9F08091AD049091AE0495
:104E80008E7F0E946D09182F6091AB048091B6044B
:104E90000E94EF13482F612F8091B50449A30E940F
:104EA000EF130091D805282F49A16091B304809198
:104EB000B4040E94F62442988091C7048130C1F066
:104EC00018F08230B1F1C8C082E10E94192A892B02
:104ED00009F0C2C081E08093C7040E94F428609367
:104EE000C3047093C4048093C5049093C604B4C0F3
:104EF00082E10E94192A892B31F50E94F428C09082
:104F0000C304D090C404E090C504F090C6046C19AA
:104F10007D098E099F09693E73408105910508F45A
:104F20009BC082E08093C70480ED97E00E94B607A3
:104F300093C082E10E94192A892B09F48DC080E078
:104F400090E00E94B6071092C70486C080E090E00F
:104F50000E94B607F9CE68E016CF851709F416CF80
:104F60004F5F242F30E090E0F901EE58FB4FDC0159
:104F7000A75BBB4F7C917083F901E05CFB4F7083B2
:104F800001968F7101CF2430B1F42091400481E467
:104F900094E0A3E7B4E0FC013E2F381B321718F46D
:104FA00031913D93F9CF87E3820F90917204892B61
:104FB00080937204F6CE8091C704823051F49160E0
:104FC00090937204439A8E010F5F1F4FF12CB8012A
:104FD00010C0439880913D04811103C081E080930B
:104FE0003D0480913D04833071F784E080933D045B
:104FF000EACF8F2D69A37AA30E941816F801819336
:1050000091938F01F39469A17AA1F0E1FF12F1CF9E
:105010008091A20543E754E087700E94BC08C4CE8B
:10502000882309F4C8CE2091C80431E0320F3093B0
:10503000C8042913C0CE0CC01092CA04DCCE8091E3
:10504000AA04883009F4439A89E08093AA04D3CE55
:105050001092C8048150AFCEA296ECE00C94BB2E07
:105060008230E8F4E82FF0E0EE0FFF1FE752FA4F2E
:1050700071836083813041F0809169008C7F842B43
:1050800080936900E89A089580916900440F551F44
:10509000440F551F837F842B80936900E99A0895FC
:1050A0001F920F920FB60F9211242F933F934F939D
:1050B0005F936F937F938F939F93AF93BF93EF9380
:1050C000FF938091D9059091DA05892B29F0E09121
:1050D000D905F091DA050995FF91EF91BF91AF9154
:1050E0009F918F917F916F915F914F913F912F9100
:1050F0000F900FBE0F901F9018951F920F920FB632
:105100000F9211242F933F934F935F936F937F934D
:105110008F939F93AF93BF93EF93FF938091DB05A2
:105120009091DC05892B29F0E091DB05F091DC05FD
:105130000995FF91EF91BF91AF919F918F917F91D1
:105140006F915F914F913F912F910F900FBE0F90F4
:105150001F9018951F920F920FB60F9211242F9344
:105160003F938F939F93AF93BF938091DE05909170
:10517000DF05A091E005B091E1053091DD0523E068
:10518000230F2D3720F40196A11DB11D05C026E87F
:10519000230F0296A11DB11D2093DD058093DE052E
:1051A0009093DF05A093E005B093E1058091E205BF
:1051B0009091E305A091E405B091E5050196A11D4C
:1051C000B11D8093E2059093E305A093E405B093AD
:1051D000E505BF91AF919F918F913F912F910F90D6
:1051E0000FBE0F901F9018952FB7F8946091DE05B1
:1051F0007091DF058091E0059091E1052FBF089542
:105200003FB7F8948091E2059091E305A091E40501
:10521000B091E50526B5A89B05C02F3F19F0019672
:10522000A11DB11D3FBF6627782F892F9A2F620FCE
:10523000711D811D911D42E0660F771F881F991F08
:105240004A95D1F70895CF92DF92EF92FF92CF93D4
:10525000DF936B017C010E940029EB01C114D10492
:10526000E104F10479F00E9400296C1B7D0B683E7B
:105270007340A0F381E0C81AD108E108F108C851D1
:10528000DC4FECCFDF91CF91FF90EF90DF90CF908C
:105290000895789484B5826084BD84B5816084BDAE
:1052A00085B5826085BD85B5816085BDEEE6F0E09F
:1052B000808181608083E1E8F0E0108280818260FB
:1052C0008083808181608083E0E8F0E0808181607C
:1052D0008083E1EBF0E0808184608083E0EBF0E0AC
:1052E000808181608083EAE7F0E080818460808350
:1052F00080818260808380818160808380818068FA
:1053000080831092C1000895833081F028F48130A9
:1053100099F08230A1F008958630A9F08730B9F075
:105320008430D1F4809180008F7D03C08091800013
:105330008F7780938000089584B58F7702C084B5FD
:105340008F7D84BD08958091B0008F7703C08091D8
:10535000B0008F7D8093B0000895CF93DF9390E0ED
:10536000FC01ED50F44F2491FC01E95FF34F84916F
:10537000882349F190E0880F991FFC01E15DF34F0C
:10538000A591B4918B5D934FFC01C591D4919FB7CA
:10539000611108C0F8948C91209582238C938881A8
:1053A00082230AC0623051F4F8948C91322F3095E8
:1053B00083238C938881822B888304C0F8948C91FA
:1053C000822B8C939FBFDF91CF910895A1E0B0E035
:1053D000ECEEF9E20C94A72E282F30E0F901E1520F
:1053E000F44F8491F901ED50F44F1491F901E95F04
:1053F000F34F04910023C9F0882321F069830E94B0
:1054000084296981E02FF0E0EE0FFF1FEB5DF34F81
:10541000A591B4919FB7F8948C91611103C0109538
:10542000812301C0812B8C939FBF2196E4E00C94D3
:10543000C32ECF93DF93282F30E0F901E152F44FD0
:105440008491F901ED50F44FD491F901E95FF34FE4
:10545000C491CC2391F081110E948429EC2FF0E0BB
:10546000EE0FFF1FE55EF34FA591B4912C912D2314
:1054700081E090E021F480E002C080E090E0DF91E4
:10548000CF9108958E3008F08E50877020919D0145
:1054900090E4299F90011124822B80937C008091BD
:1054A0007A00806480937A0080917A0086FDFCCF38
:1054B000809178002091790090E0922B0895A0E0EF
:1054C000B0E0E5E6FAE20C94A32E6C017A01EB0160
:1054D000E60EF71E00E010E0CE15DF0561F06991E1
:1054E000D601ED91FC910190F081E02DC601099566
:1054F000080F191FF1CFC801CDB7DEB7E8E00C9453
:10550000BF2E6115710589F0DB010D900020E9F7D0
:10551000AD0141505109461B570BDC01ED91FC9147
:105520000280F381E02D0995089580E090E00895D0
:10553000EF92FF920F931F93CF93DF938C01FB01A8
:10554000C0E0D0E064917F018FEFE81AF80A66238B
:1055500061F0D801ED91FC910190F081E02DC8013E
:105560000995C80FD91FF701EDCFCE01CDB7DEB732
:10557000E6E00C94C12E0E94812A0895DC01ED9191
:10558000FC910190F081E02D099508950F931F93F0
:10559000CF93DF93EC016DE00E94BE2A8C016AE09C
:1055A000CE010E94BE2A800F911FDF91CF911F91E3
:1055B0000F9108950F931F93CF93DF93EC010E94F7
:1055C000982A8C01CE010E94C62A800F911FDF917C
:1055D000CF911F910F9108950F931F93CF93DF9356
:1055E000EC010E94812A8C01CE010E94C62A800F04
:1055F000911FDF91CF911F910F9108950F931F93EA
:10560000CF93DF93EC010E94BE2A8C01CE010E9451
:10561000C62A800F911FDF91CF911F910F9108959E
:10562000A1E2B0E0E6E1FBE20C949F2E7C01C42EE7
:10563000E52FCB01D22E19A221E02D1510F02AE082
:10564000D22E8E010F5D1F4F8D2C912CA12CB12CD1
:105650006C2D7E2FA50194010E94582E8C2DD29E78
:1056600080191124015011098A3010F4805D01C0A5
:10567000895CF8018083211531054105510521F030
:10568000C22EE32FCA01E4CFB801C7010E94812ACC
:10569000A196ECE00C94BB2EA0E0B0E0E2E5FBE2CA
:1056A0000C94A32EEC016A017B012115310541F414
:1056B000E881F9810190F081E02D642F09951DC0EA
:1056C0002A303105A9F477FF12C06DE20E94BE2A8C
:1056D0008C0144275527BA014C195D096E097F09D1
:1056E0002AE0CE010E94102B800F911F06C02AE0F5
:1056F000B701A601CE010E94102BCDB7DEB7E8E0BE
:105700000C94BF2E9A01AB01662757FD6095762F4A
:105710000E944C2B08950F931F93CF93DF93EC01BE
:105720009A01AB01662757FD6095762F0E944C2B9E
:105730008C01CE010E94C62A800F911FDF91CF916C
:105740001F910F9108952115310549F4DC01ED9168
:10575000FC910190F081E02D642F099508950E943D
:10576000102B08959A01462F50E060E070E00E94EF
:10577000A32B08959A01AB0160E070E00E94A32B77
:1057800008950F931F93CF93DF93EC010E94A32BF7
:105790008C01CE010E94C62A800F911FDF91CF910C
:1057A0001F910F9108950F931F93CF93DF93EC01F7
:1057B0009A01AB0160E070E00E94A32B8C01CE0146
:1057C0000E94C62A800F911FDF91CF911F910F91E8
:1057D00008950F931F93CF93DF93EC019A01462F07
:1057E00050E060E070E00E94A32B8C01CE010E948B
:1057F000C62A800F911FDF91CF911F910F910895BD
:10580000FC0124853585F901E05CFF4F80819181A1
:10581000F901EE5BFF4F20813181821B930B8F7367
:1058200099270895FC0184859585FC01E05CFF4F74
:1058300040815181FC01EE5BFF4F20813181421795
:10584000530741F00190F081E02DE80FF91F8081AE
:1058500090E008958FEF9FEF0895FC018485958572
:10586000FC01E05CFF4F40815181FC01EE5BFF4F8A
:10587000208131814217530779F0A081B181A80FAF
:10588000B91F8C91208131812F5F3F4F2F733327B8
:105890003183208390E008958FEF9FEF0895FC01FE
:1058A00081A1882329F0A489B5898C9186FFFBCF3B
:1058B00011A20895CF93DF93FC0126853785D90186
:1058C000A05CBF4F8D919C91119701968F73992782
:1058D000E901CE5BDF4F4881598184179507D9F3E1
:1058E0000D90BC91A02DA20FB31F6C93A685B78518
:1058F000A05CBF4F11969C938E93A689B7892C917B
:1059000081E090E0078C02C0880F991F0A94E2F7AB
:10591000282B2C9381E081A30488F589E02D8081D8
:105920008064808381E090E0DF91CF9108950895B5
:105930001F920F920FB60F9211242F933F934F9304
:105940008F939F93EF93FF938091C00082FD1CC0C3
:105950004091C60080918C0690918D0601968F73C0
:10596000992720918E0630918F068217930771F048
:10597000E0918C06F0918D06E45BF94F40839093A3
:105980008D0680938C0602C08091C600FF91EF9136
:105990009F918F914F913F912F910F900FBE0F903C
:1059A0001F90189586EE95E00E94002C892B11F02F
:1059B0000E94972C08951F920F920FB60F921124F8
:1059C0002F933F938F939F93EF93FF9320914806DC
:1059D0003091490680914A0690914B062817390765
:1059E00031F48091C1008F7D8093C10014C0E0919B
:1059F0004A06F0914B06E85FF94F208180914A06F4
:105A000090914B0601968F73992790934B06809344
:105A10004A062093C600FF91EF919F918F913F918D
:105A20002F910F900FBE0F901F901895A0E0B0E03F
:105A3000ECE1FDE20C949F2EFC011382128288EEB1
:105A400093E0A0E0B0E084839583A683B7838CEBDA
:105A500093E0918380837587648757874687318B6E
:105A6000208B138B028BF58AE48AD78AC68AB18E83
:105A7000A08E938E828E8F85848F8889858F898969
:105A8000868F8A89878F8B8980A3ECE00C94BB2E4C
:105A9000CF92DF92EF92FF92CF93DF93EC016A01F6
:105AA0007B01411581EE580761057105F9F0EC891C
:105AB000FD8981E090E008A002C0880F991F0A9438
:105AC000E2F7808360E079E08DE390E0A701960142
:105AD0000E94582E21503109410951095695479588
:105AE00037952795211580E1380798F0EC89FD89D5
:105AF000108260E874E88EE190E0A70196010E94B0
:105B0000582E21503109410951095695479537952D
:105B10002795E889F9893083EA89FB89208319A2CE
:105B2000EE89FF89408181E090E09C010C8C02C0ED
:105B3000220F331F0A94E2F7422B4083EE89FF893C
:105B400040819C010D8C02C0220F331F0A94E2F7A2
:105B5000422B4083EE89FF8940819C010E8C02C05C
:105B6000220F331F0A94E2F7422B4083EE89FF890C
:105B700020810F8C02C0880F991F0A94E2F780954C
:105B800082238083DF91CF91FF90EF90DF90CF90C1
:105B900008958F929F92AF92BF92CF92DF92EF9231
:105BA000FF920F931F9381E08F9385E08F9387E09F
:105BB0008F9383E08F9384E08F93E6EC8E2E912C6D
:105BC000F2ECAF2EB12CA1ECCA2ED12CB0ECEB2E06
:105BD000F12C04EC10E025EC30E048E056E06CE4F9
:105BE00076E086EE95E00E94162D0F900F900F90B4
:105BF0000F900F901F910F91FF90EF90DF90CF903B
:105C0000BF90AF909F908F9008950E9449290E9465
:105C1000B522C2EDDCE20E9449252097E1F30E9403
:105C2000D22CF9CFA29FB001B39FC001A39F700DEA
:105C3000811D1124911DB29F700D811D1124911D94
:105C400008950E94122EA59F900DB49F900DA49FC1
:105C5000800D911D11240895B7FF0C94212E0E94F0
:105C6000212E821B930B0895DB018F939F930E943B
:105C7000212EBF91AF91A29F800D911DA39F900DEA
:105C8000B29F900D1124089597FB072E16F40094EF
:105C900007D077FD09D00E94D62E07FC05D03EF430
:105CA000909581959F4F0895709561957F4F0895C8
:105CB000A1E21A2EAA1BBB1BFD010DC0AA1FBB1F10
:105CC000EE1FFF1FA217B307E407F50720F0A21B82
:105CD000B30BE40BF50B661F771F881F991F1A94EF
:105CE00069F760957095809590959B01AC01BD0119
:105CF000CF010895052E97FB1EF400940E94912E6B
:105D000057FD07D00E94582E07FC03D04EF40C9488
:105D1000912E50954095309521953F4F4F4F5F4FB5
:105D2000089590958095709561957F4F8F4F9F4F07
:105D300008952F923F924F925F926F927F928F922F
:105D40009F92AF92BF92CF92DF92EF92FF920F930A
:105D50001F93CF93DF93CDB7DEB7CA1BDB0B0FB614
:105D6000F894DEBF0FBECDBF09942A8839884888D1
:105D70005F846E847D848C849B84AA84B984C88467
:105D8000DF80EE80FD800C811B81AA81B981CE0F5E
:105D9000D11D0FB6F894DEBF0FBECDBFED01089543
:105DA000EE0FFF1F0590F491E02D0994AA1BBB1B79
:105DB00051E107C0AA1FBB1FA617B70710F0A61B0B
:105DC000B70B881F991F5A95A9F780959095BC012C
:105DD000CD0108958F929F92AF92BF92CF92DF92A2
:105DE000EF92FF92CF93DF93EC01688179818A81F2
:105DF0009B81611571058105910521F464E279EDBE
:105E00008BE597E02DE133EF41E050E00E947A2EE0
:105E100049015A019B01AC01A7EAB1E40E94212E7D
:105E20006B017C01ACEEB4EFA50194010E942F2E12
:105E3000C60ED71EE81EF91EF7FE06C081E0C81A7E
:105E4000D108E10880E8F80AC882D982EA82FB8298
:105E5000C701B6019F77DF91CF91FF90EF90DF9060
:105E6000CF90BF90AF909F908F9008950E94EA2EA0
:105E7000089586E091E00E94EA2E0895609306015D
:105E800070930701809308019093090108952F9260
:105E90003F925F926F927F928F929F92AF92BF924A
:105EA000CF92DF92EF92FF920F931F93CF93DF93E6
:105EB0008B01EA016115710521F0DB018C931196CC
:105EC0009C93209739F09E012250310923323105ED
:105ED00008F0D8C07C016701BFEFCB1ADB0A56017E
:105EE000F7016080862D90E00E947930892B11F0B7
:105EF0007601F1CFFDE26F120AC0570182E0A80ED1
:105F0000B11CD70111966C90772473940BC0BBE23F
:105F10006B1207C05701E2E0AE0EB11CD70111961B
:105F20006C90712CCE018F7E892B89F4B0E36B12BB
:105F300037C0F50180818F7D8835D1F46180F2E032
:105F4000AF0EB11C872D8260782EC0E1D0E0CA3040
:105F5000D10551F1C031D10521F0C830D10599F4F6
:105F600009C0CC24CA94DC2CEC2CAFE0FA2E22C061
:105F7000209769F7C8E0D0E0CC24CA94DC2CEC2C44
:105F8000FFE1FF2E17C06FEF7FEFCB019E0144278B
:105F900037FD4095542F0E94582E69017A010AC09E
:105FA0002097A9F6CAE0D0E0E9E9CE2EDC2CEC2C53
:105FB000E9E1FE2EF50160E020E030E0A9014E01AC
:105FC000AA2497FCA094BA2C1F0170ED572E560CF2
:105FD000A9E0A51570F48FEB860D8A3118F499ECC1
:105FE000592E06C08FE9860D8A3148F589EA582E68
:105FF000560C852D90E08C179D070CF56F3FD9F05E
:10600000C216D306E406F50698F0C501B4010E9455
:10601000342E9B01AC01852D90E0A0E0B0E0280F6C
:10602000391F4A1F5B1F281739074A075B0710F4FF
:106030006FEF01C061E03196D1016C90C5CF0115C1
:10604000110551F0662311F0319703C071FE04C0B1
:106050003297D801ED93FC9370FE07C050954095A0
:10606000309521953F4F4F4F5F4F67FF10C082E241
:1060700090E090939106809390066FEF7FEF8FEF03
:106080009FEF07C060E070E080E090E002C0B901DF
:10609000CA01DF91CF911F910F91FF90EF90DF9098
:1060A000CF90BF90AF909F908F907F906F905F90B8
:1060B0003F902F900895FC0188279927E89421911B
:1060C0002032E9F3293010F02E30C8F32B3241F0A2
:1060D0002D3239F4689404C00E94AD30820F911DB6
:1060E000219120532A30C0F31EF4909581959F4F43
:1060F0000895911150C0803219F089508550D0F721
:10610000089548EC53E00E9486300895FA01A19169
:10611000B081009719F41097E1F0CD01DC01CD01B9
:106120000D90002011F4C00113C0FB012191222326
:1061300019F02015D9F7F3CFFB012191201519F49F
:106140001E92119606C02223C1F70D900020A1F7E0
:10615000D001FA01A193B08308957AE0979F902D22
:10616000879F802D910D11240895F999FECF92BD3E
:1061700081BDF89A992780B50895262FF999FECF09
:106180001FBA92BD81BD20BD0FB6F894FA9AF99A54
:106190000FBE01960895992788270895F894FFCF98
:1061A00000009206200001000000FF000200020033
:1061B00002000200020002000200020002000200CF
:1061C0000200020002000200020002802500000519
:1061D000400AA1204EA50020244EA52C2330C01239
:1061E00000001A400AA1204EA5001B1E27522C2396
:1061F000308025000005400AA1204EA50020244E35
:10620000A52C2330004B000006400AD0009D490019
:106210007B289D492C233000E1000005400A450100
:10622000D7DC03B81E0EBF00232E48E801008A40C9
:106230000A6001555502AD1E20000023C8015458C4
:106240002074696D656F75742100596573004E6F18
:10625000002C00386368004E2F41002C205B005D4D
:106260002028002900486F70206368616E6E656C9D
:10627000200020402000456E746572696E672061C1
:1062800064617074697665206368616E6E656C2008
:1062900073656C656374696F6E2C207069636B69DC
:1062A0006E673A007363616E6E6572206D6F646530
:1062B000004E4F5420454E41424C45440053656EBC
:1062C00064696E672073657474696E677320746F98
:1062D0002052580A00526573657474696E672073A2
:1062E000657474696E6773206F6E2052580A00419E
:1062F000626F727465642065646974730A00696E04
:1063000076616C69642073656C656374696F6E0097
:106310000D0A496E76616C696420696E707574202F
:106320002D2064697363617264656421070053659D
:106330007474696E677320736176656420746F206E
:10634000454550524F4D0A0052657665727465643A
:106350002073657474696E67732066726F6D204573
:106360004550524F4D0A004C6F6164656420666170
:1063700063746F72792064656661756C74730A006A
:106380004B657920616E64206368616E6E656C7325
:106390002072616E646F6D697A65640A004F706582
:1063A0006E4C52536E672054582073746172746936
:1063B0006E672000206F6E20485720006D6F647557
:1063C0006C65206C6F636B65643F00342B34003860
:1063D00000382B340031320031322B34003136009A
:1063E00050504D0052535349005344410053434CC5
:1063F00000525844005458440041494E004C424514
:1064000045500053504B54524D0053425553005386
:10641000554D44004C4C494E440000070B0C1011E4
:106420001500B7012B032F033103350338033D0358
:10643000B7014003440349034D0351035503590376
:106440005D0363036A036F0374038D028D028D0283
:106450008D02160A13223129000000005A2C5F2AEF
:08646000002C2D2C122C4F2CF6
:107E00000F92CDB7DEB7112484B714BE81FFF1D035
:107E100082E08093C00088E18093C10086E0809377
:107E2000C20080E18093C4008EE0CDD088249924E4
:107E3000CC24C394F5E0DF2EE1E1EE2E73E0F72EC3
:107E4000B6D0082F813479F4B2D08983C2D0898129
:107E5000823811F481E005C0813811F485E001C059
:107E600083E09ED09AC0823411F484E103C085344B
:107E700019F485E0B6D091C0853561F498D0082F0B
:107E800010E095D090E0982E8824802A912A880CC2
:107E9000991C82C0863521F484E0A3D080E0E1CF34
:107EA000843609F04CC083D082D0A82E80D0B82E62
:107EB00000E011E07CD0F80181938F01AE16D1F77C
:107EC00088D0FB2DF53489F4E0E0F1E00BC0F9999E
:107ED000FECF92BC81BC0894811C911C819180BD15
:107EE000FA9AF99AEA1598F358C08B2D863409F05E
:107EF00054C0F401F7BEE89507B600FCFDCFF401CD
:107F0000A0E0B1E02C9130E011968C91119790E0B7
:107F1000982F8827822B932B12960C01C7BEE895C9
:107F20001124329681E0A038B80761F7F401D7BE7A
:107F3000E89507B600FCFDCFE7BEE8952EC0843774
:107F4000F1F435D034D0182F32D0B82E42D0FB2DDA
:107F5000F63421F4F40105914F010CC0FB2DF534EA
:107F600049F4F999FECF92BC81BC0894811C911C04
:107F7000F89A00B5802F14D0115049F70EC08537FC
:107F800039F427D08EE10CD085E90AD08FE069CF93
:107F9000813511F488E017D01CD080E101D050CF9A
:107FA0009091C00095FFFCCF8093C600089580910A
:107FB000C00087FFFCCF8091C00084FD01C0A89560
:107FC0008091C6000895E0E6F0E098E19083808318
:107FD0000895EDDF803219F088E0F5DFFFCF84E10E
:107FE000DFCF1F93182FE3DF1150E9F7F2DF1F9166
:0E7FF0000895282E80E0E7DFEE27FF27099492
:027FFE0001057B
:0400000300007E007B
:00000001FF
